:100000001c9c048405a51dbd808560840000001a29
:100010001b5b1a1b609ae08405e0a40586c084007f
:10002000a6e00282004000036200424000820062bb
:100030008482004000e0008403620042400244e009
:10004000008402e0440242e042820040400560a297
:10005000848300606002e040040402e04402e04463
:10006000bdbfb0bda4a2a3a5b0b1b2a7b4b5b6b789
:1000700000a64003630242626002820040024282a4
:10008000000400048200400400840000028200009a
:10009000020283424340000004820042830244641f
:1000a000408260820400840000000082005042828e
:1000b000a4a2a3a5b0b1b2a7b4b5b6b7a6bdbf40c0
:1000c000bd00bfb0e0bd060404c3e0c5820044002b
:1000d00083830062826400836382426260028200e2
:1000e0008200420040008000008200430083428280
:1000f000e000bdbfb090820040420010500260831b
:10010000004350828240820042424010000000bf03
:10011000b0e0bdbdbfb2b1b0900003630242626007
:1001200000000000004002020011820040424363d0
:10013000424262601200800000120000222284000d
:10014000824363424262600020bfb2b1b0e0bdbdf5
:10015000bfb100b000409000000000400202024029
:1001600002020000000202000000230000006023e1
:100170000701610121000600000060230701610101
:10018000210006008400836382426260028220bff5
:10019000b1b0e0bdbdbfb0820042424002000000ed
:1001a00000830062000000000040830262040084bb
:1001b000000000008200400004008400bfb0e0bde9
:1001c0008082004080a5a20040a5a500a5c2a30092
:1001d000c3a2c6a5c54000e080bd81bf02a2a504a0
:1001e00080a008088800090462c006460282c2e2b4
:1001f0006080e7a702a2a7e000a0bf00e0bdbdbfee
:10020000b1b0101090000000004004008400000411
:100210000084002004008485002084000004008401
:10022000bfb1b0e0bda200404083a5a3006084e060
:1002300080bdbf800400840000bf00e0bdbdbfb032
:10024000000302426202428204008404008404002b
:100250008404008404008404008404008404008472
:1002600004008404008404008404008482004000ac
:100270008000100240000400840000020363430277
:100280004282e000bdbf0242820000bf00e0bdbd6f
:10029000bf04008400bf00e0bd0000000000004576
:1002a00072006f2072770a20737220756400004814
:1002b0002000440a2a0030312d3528292d332933d6
:1002c0000031332d2933330a33340030342d2932b1
:1002d0000a2d3333312931332833003333336673f6
:1002e000000000000000000000000000000000000e
:1002f00000000000000000000000000000000000fe
:1003000000000000000000000000000000000000ed
:00000001ff
